S01E000062696E2F64656D6F70726F675F73746D3332663330332E737265632D
S3150800400000A00020F9420008494300084943000877
S3150800401049430008494300084943000800000000D6
S3150800402000000000000000000000000049430008EE
S31508004030494300080000000049430008294F0008CA
S315080040404943000849430008494300084943000812
S315080040504943000849430008494300084943000802
S3150800406049430008494300084943000849430008F2
S3150800407049430008494300084943000849430008E2
S3150800408049430008494300084943000849430008D2
S3150800409049430008494300084943000849430008C2
S315080040A049430008494300084943000849430008B2
S315080040B049430008494300084943000849430008A2
S315080040C04943000849430008494300084943000892
S315080040D04943000849430008494300084943000882
S315080040E04943000849430008494300084943000872
S315080040F04943000849430008494300084943000862
S31508004100000000000000000000000000494300080D
S315080041104943000849430008494300084943000841
S315080041204943000849430008494300084943000831
S315080041304943000849430008000000000000000049
S3150800414049430008494300084943000800000000A5
S315080041500000000000000000000000000000000051
S315080041600000000000000000494300084943000819
S31508004170494300080000000000000000000000009D
S311080041800000000049430008EE11AA5593
S3150800418C10B5054C237833B9044B13B10448AFF377
S3150800419C00800123237010BD3004002000000000AD
S315080041AC1051000808B5034B1BB103490348AFF37C
S315080041BC008008BD000000003404002010510008DF
S315080041CC70B50D4E0D4D761BB61006D00024013475
S315080041DC55F8043B9847A642F9D1094E094D761B6A
S315080041EC00F090FFB61006D00024013455F8043BB5
S315080041FC9847A642F9D170BD5C5100085C5100087D
S3150800420C645100085C510008024B13B1024800F0D7
S3150800421C05B8704700000000354200080023014627
S3150800422C1A46184600F01EB838B50A4C0A4D641BD7
S3150800423CA4100AD004F18043013B05EB8305013C2D
S3150800424C55F804399847002CF9D1BDE8384000F0E8
S3150800425C5FBF00BF6851000864510008704700BF73
S3150800426C704700BF2DE9F0411E4C05462068904664
S3150800427C1F460E46FFF7F2FF1B4B1A68D2F8483159
S3150800428C33B35A6820681F2A27DC4DB9911C0132B2
S3150800429C5A6043F82160FFF7E3FF0020BDE8F08180
S315080042AC03EB82010124C1F8888004FA02FED3F8D4
S315080042BC8841022D44EA0E0CC3F888C1C1F808716E
S315080042CCE4D1D3F88C114EEA0104C3F88C41DDE72E
S315080042DC02F5A673C2F84831D3E7FFF7C1FF4FF0D2
S315080042ECFF30DBE72804002028510008DFF834D01B
S315080042FC002103E00C4B5B58435004310B480C4B24
S3150800430C42189A42F6D30B4A02E0002342F8043BC1
S3150800431C094B9A42F9D300F0B3FDFFF751FF00F0B1
S3150800432C72FEFEE700A0002068510008000000207D
S3150800433C30040020300400207C040020FEE7000036
S3150800434C074AD36823F4E0631B041B0C000200F431
S3150800435CE060184340F0BF6040F40030D06070470E
S3150800436C00ED00E030B4174BDB68C3F30223C3F14E
S3150800437C0704042C28BF04241D1D062D01D9033B54
S3150800438C00E000234FF0FF3505FA04F421EA040196
S3150800439C994005FA03F322EA03031943002809DBBB
S315080043AC0901C9B200F1604000F5614080F80013BC
S315080043BC30BC704700F00F000901C9B2024B195402
S315080043CCF6E700BF00ED00E014ED00E00138B0F1AF
S315080043DC807F0AD2064B5860064AF02182F82310D1
S315080043EC0020986007221A6070470120704700BFAA
S315080043FC10E000E000ED00E0042805D0054A13683B
S3150800440C23F0040313607047024A136843F004034D
S3150800441C1360704710E000E0704708B5FFF7FCFF23
S3150800442C08BD0000F0B482B0002336E0042400E096
S3150800443C0024B4403C4302355B4E46F825405B4CA1
S3150800444C2568D44304EA05064F6817F4803F01D063
S3150800445C42EA0506554D2E606D6804EA05064F6856
S3150800446C17F4003F01D042EA0506504D6E60AD6860
S3150800447C04EA05064F6817F4801F01D042EA0506C0
S3150800448C4A4DAE60ED682C404E6816F4001F01D0FC
S3150800449C42EA0504454AD46001330A6832FA03F441
S315080044AC7ED001249C402240F6D04D68022D01D0C6
S315080044BC122D10D1DE08083650F826C003F0070571
S315080044CCAF000F25BD402CEA050C0D69BD4045EA29
S315080044DC0C0540F8265006685F000325BD40ED43E1
S315080044EC05EA060C4E6806F00306BE4046EA0C06BC
S315080044FC06604E6806F1FF3CBCF1010F03D9112E7C
S3150800450C01D0122E10D1866805EA060CCE68BE407C
S3150800451C46EA0C068660466826EA04044E68C6F324
S3150800452C00169E4026434660C46825408C68BC40ED
S3150800453C2C43C4604C6814F0805FADD01C4CA56944
S3150800454C45F00105A561A46904F001040194019CD8
S3150800455C9D08AE1C144C54F8267003F00304A600F0
S3150800456C0F24B44027EA0407B0F1904F3FF460AF2C
S3150800457C104CA0420ED004F58064A0420CD004F571
S3150800458C8064A0420AD004F58064A0423FF44EAF82
S3150800459C05244EE701244CE702244AE7032448E79E
S315080045AC02B0F0BC704700BF000001400004014097
S315080045BC00100240000400480AB18161704781620C
S315080045CC7047000010B50446074B1868074BA3FB49
S315080045DC00308009FFF7FAFE002221464FF0FF3023
S315080045ECFFF7C0FE002010BD2C040020D34D62102E
S315080045FC08B5074A136843F0100313600320FFF746
S3150800460C9FFE0020FFF7DEFF00F004FD002008BD2A
S3150800461C00200240024A136801331360704700BF3A
S3150800462C78040020014B1868704700BF78040020F6
S3150800463C70B582B00446036813F0010F3BD0B54B36
S3150800464C5B6803F00C03042B1ED0B24B5B6803F0BB
S3150800465C0C03082B13D06368B3F5803F68D0002B86
S3150800466C40F0928003F1804303F504331A6822F470
S3150800467C80321A601A6822F480221A605DE0A54B13
S3150800468C5B6813F4803FE6D04FF4003393FAA3F338
S3150800469CA04B19684FF4003393FAA3F3B3FA83F3D8
S315080046AC03F01F03012202FA03F30B4203D06368DB
S315080046BC002B00F0A782236813F0020F00F0C580C8
S315080046CC944B5B6813F00C0F00F09C80914B5B6865
S315080046DC03F00C03082B00F08F802369002B00F0E5
S315080046ECF280012292FAA2F3B3FA83F303F184530C
S315080046FC03F584139B001A60FFF794FF0546022303
S3150800470C93FAA3F3834B1968022393FAA3F3B3FA28
S3150800471C83F303F01F03012202FA03F30B4240F062
S3150800472CC380FFF77FFF401B0228E8D9032072E2FB
S3150800473C784A136843F480331360764AD36A23F0B5
S3150800474C0F03A1680B43D3626368002B36D0FFF7BF
S3150800475C69FF05464FF4003393FAA3F36D4B1968BA
S3150800476C4FF4003393FAA3F3B3FA83F303F01F035E
S3150800477C012202FA03F319429DD1FFF753FF401B9E
S3150800478C6428E7D9032046E2B3F5A02F09D0614B7C
S3150800479C1A6822F480321A601A6822F480221A6087
S315080047ACCBE703F18043A3F53C331A6842F4802225
S315080047BC1A601A6842F480321A60BEE7FFF732FFB5
S315080047CC05464FF4003393FAA3F3524B19684FF48A
S315080047DC003393FAA3F3B3FA83F303F01F0301220E
S315080047EC02FA03F319423FF466AFFFF71BFF401BAF
S315080047FC6428E6D903200EE2464B5B6813F4803F27
S3150800480C7FF46BAF022393FAA3F3424B1968022386
S3150800481C93FAA3F3B3FA83F303F01F03012202FA04
S3150800482C03F3194203D02369934240F0ED813948CA
S3150800483C036823F0F8036169F82292FAA2F2B2FA35
S3150800484C82F201FA02F213430360236813F0080F8D
S3150800485C00F08C80A369002B60D0012191FAA1F29B
S3150800486CB2FA82F22C4B13449B001960FFF7DAFE5E
S3150800487C0546022393FAA3F293FAA3F293FAA3F248
S3150800488C244A516A93FAA3F3B3FA83F303F01F038A
S3150800489C012202FA03F30B4268D1FFF7C3FE401B51
S315080048AC0228E6D90320B6E11A48036823F0F80370
S315080048BC6169F82292FAA2F2B2FA82F201FA02F2CB
S315080048CC13430360C1E7012393FAA3F3B3FA83F303
S315080048DC03F1845303F584139B0000221A60FFF737
S315080048ECA1FE0546022393FAA3F30A4B1968022381
S315080048FC93FAA3F3B3FA83F303F01F03012202FA24
S3150800490C03F31942A1D0FFF78DFE401B0228E9D903
S3150800491C032080E10010024020819010012292FAB7
S3150800492CA2F2B2FA82F2BE4B13449B0000221A6022
S3150800493CFFF778FE0546022393FAA3F293FAA3F23D
S3150800494C93FAA3F2B74A516A93FAA3F3B3FA83F329
S3150800495C03F01F03012202FA03F30B4206D0FFF7FA
S3150800496C61FE401B0228E6D9032054E1236813F0A4
S3150800497C040F00F0A980AB4BDB6913F0805F20D1E4
S3150800498CA84BDA6942F08052DA61DB6903F080538E
S3150800499C0193019B0125A44B1B6813F4807F12D04D
S315080049ACE368012B23D073BB03F1804303F504336F
S315080049BC1A6A22F001021A621A6A22F004021A62B0
S315080049CC1AE00025E7E7984A136843F480731360E6
S315080049DCFFF728FE0646944B1B6813F4807FDFD13D
S315080049ECFFF720FE801B6428F5D9032013E18D4AB6
S315080049FC136A43F001031362E368002B3CD0FFF7FC
S31508004A0C11FE06462EE0052B09D0864B1A6A22F0B3
S31508004A1C01021A621A6A22F004021A62ECE7814B46
S31508004A2C1A6A42F004021A621A6A42F001021A62FF
S31508004A3CE2E7022393FAA3F37A4B596A022393FA11
S31508004A4CA3F3B3FA83F303F01F03012202FA03F369
S31508004A5C194238D1FFF7E6FD801B41F2883398429C
S31508004A6C00F2D480022393FAA3F293FAA3F3002B51
S31508004A7CDFD06C4B196AE1E7FFF7D4FD064618E060
S31508004A8C022393FAA3F3674B596A022393FAA3F307
S31508004A9CB3FA83F303F01F03012202FA03F3194254
S31508004AAC11D0FFF7BFFD801B41F28833984200F204
S31508004ABCAF80022393FAA3F293FAA3F3002BDFD069
S31508004ACC584B196AE1E7B5BBE369002B00F0A280E5
S31508004ADC544A526802F00C02082A00F09E80022BF7
S31508004AEC2FD04FF0807393FAA3F3B3FA83F303F141
S31508004AFC845303F584139B0000221A60FFF792FD7A
S31508004B0C04464FF0007393FAA3F3464B19684FF01B
S31508004B1C007393FAA3F3B3FA83F303F01F0301228A
S31508004B2C02FA03F319426BD0FFF77CFD001B02282F
S31508004B3CE7D903206FE03B4AD36923F08053D3614E
S31508004B4CC2E74FF0807393FAA3F3B3FA83F303F136
S31508004B5C845303F584139B0000221A60FFF762FD49
S31508004B6C05464FF0007393FAA3F32E4B19684FF0D2
S31508004B7C007393FAA3F3B3FA83F303F01F0301222A
S31508004B8C02FA03F3194206D0FFF74CFD401B022824
S31508004B9CE7D903203FE023494B6823F47413626A70
S31508004BAC206A024313434B604FF0807393FAA3F3C6
S31508004BBCB3FA83F303F1845303F584139B000122A0
S31508004BCC1A60FFF72FFD04464FF0007393FAA3F310
S31508004BDC144B19684FF0007393FAA3F3B3FA83F3E3
S31508004BEC03F01F03012202FA03F3194206D1FFF759
S31508004BFC19FD001B0228E7D903200CE000200AE067
S31508004C0C002008E0012006E0012004E0032002E071
S31508004C1C032000E0002002B070BD0120FBE700BFB6
S31508004C2C208190100010024000700040164B5B6803
S31508004C3C03F00C02082A01D01448704703F47011CB
S31508004C4C4FF4701292FAA2F2B2FA82F221FA02F236
S31508004C5C0F49885C0C4AD26A02F00F020F2191FAAE
S31508004C6CA1F1B1FA81F1CA400A498A5C13F4803F72
S31508004C7C05D0064BB3FBF2F300FB03F07047064B6B
S31508004C8C03FB00F0704700BF0010024000127A00C8
S31508004C9C2C5100083C51000800093D00714B1B685B
S31508004CAC03F007038B420BD26E4A136823F00703F3
S31508004CBC0B431360136803F007038B4240F0CB8059
S31508004CCC70B5036813F0020F06D0674A536823F0D1
S31508004CDCF0038468234353600D460446036813F0B7
S31508004CEC010F7AD04368012B2FD0022B42D0022217
S31508004CFC92FAA2F25C4A1068022292FAA2F2B2FA6C
S31508004D0C82F202F01F02012101FA02F2104200F0AF
S31508004D1CA48055494A6822F0030213434B60FFF7F7
S31508004D2C81FC06466368012B39D0022B46D04E4BC4
S31508004D3C5B6813F00C0F50D0FFF774FC801B41F224
S31508004D4C88339842F3D9032084E04FF4003292FA60
S31508004D5CA2F2454A10684FF4003292FAA2F2B2FA5D
S31508004D6C82F202F01F02012101FA02F20242D0D1AC
S31508004D7C01206FE04FF0007292FAA2F23A4A1068DC
S31508004D8C4FF0007292FAA2F2B2FA82F202F01F0205
S31508004D9C012101FA02F21042BBD101205AE0324B32
S31508004DAC5B6803F00C03042B17D0FFF73BFC801B46
S31508004DBC41F288339842F2D903204BE02A4B5B68C0
S31508004DCC03F00C03082B08D0FFF72CFC801B41F2D0
S31508004DDC88339842F2D903203CE0224B1B6803F037
S31508004DEC0703AB420AD91F4A136823F007032B4360
S31508004DFC1360136803F00703AB4230D1236813F032
S31508004E0C040F06D0184A536823F4E063E1680B4391
S31508004E1C5360236813F0080F07D0134A536823F41A
S31508004E2C6053216943EAC1035360FFF7FFFE0E4B3B
S31508004E3C5B6803F0F003F02292FAA2F2B2FA82F25D
S31508004E4CD3400A4AD35CD840094B18600020FFF7B8
S31508004E5CB9FB002070BD012070470120FAE701203C
S31508004E6CF8E700BF00200240001002404C51000831
S31508004E7C2C040020014B1868704700BF2C04002036
S31508004E8C1549D1F8883043F47003C1F88830134BB0
S31508004E9C1A6842F001021A605868114A02405A60B0
S31508004EAC1A6822F0847222F480321A601A6822F484
S31508004EBC80221A605A6822F4FE025A60DA6A22F0D4
S31508004ECC0F02DA62186B074A02401A6300229A60CC
S31508004EDC4FF000638B60704700ED00E00010024055
S31508004EEC0CC07FF8CCFC00FF08B5FFF7C3FF084BD6
S31508004EFCA3FB00308009FFF769FA0420FFF77CFA58
S31508004F0C002211464FF0FF30FFF72CFA08BD00BF00
S31508004F1CD34D621008B5FFF785FB08BD08B5FFF73A
S31508004F2C79FBFFF77AFA08BD08B500224FF48071B1
S31508004F3C0148FFF741FB08BD0010004810B5FFF704
S31508004F4CE9FF0F4B1B68C31AB3F5FA7F0DD304465A
S31508004F5C0C4B1B7853B901220A4B1A704FF480710B
S31508004F6C0948FFF729FB064B1C6010BD0022054BB0
S31508004F7C1A704FF480710448FFF71EFBF3E700BF65
S31508004F8C500400204C04002000100048014A024B33
S31508004F9C9A6070470040000800ED00E000B591B03B
S31508004FAC012306934FF4A0220792002208920A9333
S31508004FBC02230D934FF480330E934FF4E0130F93A3
S31508004FCC06A8FFF735FB00B1FEE70F230193022174
S31508004FDC0291002303934FF480620492059301A86F
S31508004FECFFF75CFE00B1FEE711B05DF804FB08B5EF
S31508004FFCFFF7CCFFFFF7FCFAFFF7D0FFFFF774FFBC
S3150800500CFFF792FF08BD08B5FFF7F1FFFFF796FF0C
S3150800501CFCE7000070B58AB0384B9A6942F0010279
S3150800502C9A619A6902F001020192019A5A6942F44C
S3150800503C80025A615A6902F480020292029A5A69EB
S3150800504C42F400125A615A6902F400120392039A46
S3150800505C5A6942F400325A615B6903F400330493CB
S3150800506C049B0320FFF76CF9002211466FF00B0026
S3150800507CFFF778F9002211466FF00A00FFF772F96C
S3150800508C002211466FF00900FFF76CF90022114651
S3150800509C6FF00400FFF766F9002211466FF0030063
S315080050ACFFF760F9002211466FF00100FFF75AF975
S315080050BC002211464FF0FF30FFF754F94FF4805693
S315080050CC059601250695002407940323089305A93C
S315080050DC4FF09040FFF7A6F9224631464FF0904024
S315080050ECFFF76AFA4FF480730593069507940894AC
S315080050FC05A90348FFF796F90AB070BD00100240DF
S3150800510C00100048F8B500BFF8BC08BC9E467047AE
S3110800511CF8B500BFF8BC08BC9E467047FA
S315080051280000002002030405060708090A0B0C0DEF
S315080051380E0F10100102030405060708090A0B0CCE
S315080051480D0E0F1000000000000000000102030405
S309080051580607080927
S30D0800515C15420008B1410008E4
S309080051648D41000863
S3150800516800000000EC02002054030020BC030020C5
S315080051780000000000000000000000000000000019
S315080051880000000000000000000000000000000009
S3150800519800000000000000000000000000000000F9
S315080051A800000000000000000000000000000000E9
S315080051B800000000000000000000000000000000D9
S315080051C800000000000000000000000000000000C9
S315080051D800000000000000000000000000000000B9
S315080051E800000000000000000000000000000000A9
S315080051F80000000000000000000000000000000099
S315080052080000000000000000010000000000000087
S315080052180E33CDAB34126DE6ECDE05000B0000004C
S315080052280000000000000000000000000000000068
S315080052380000000000000000000000000000000058
S315080052480000000000000000000000000000000048
S315080052580000000000000000000000000000000038
S3150800558800000000000000005404002000127A0001
S705080042F9B7
